:020000040800F2
:1000000000060020E1020008E3020008E302000805
:10001000E3020008E3020008E3020008E30200082C
:10002000E3020008E3020008E3020008253B0008A1
:10003000E3020008E3020008E3020008E30200080C
:10004000E3020008E3020008E3020008E3020008FC
:10005000E3020008E30200080D3F0008393F0008F2
:10006000653F0008913F0008BD3F0008E30200081B
:10007000E3020008E3020008E3020008E3020008CC
:10008000E3020008E3020008E3020008E3020008BC
:10009000E3020008E3020008E3020008E93F000869
:1000A000E3020008E3020008E3020008E30200089C
:1000B000E3020008E3020008E3020008E30200088C
:1000C000E3020008E3020008E3020008E30200087C
:1000D000E3020008E3020008E3020008E30200086C
:1000E0004D400008E3020008E3020008E3020008B4
:1000F000E3020008E3020008E3020008E30200084C
:10010000E3020008E3020008D5400008E30200080B
:10011000E3020008E3020008E3020008E30200082B
:10012000E3020008E3020008E3020008E30200081B
:10013000E3020008E3020008E3020008E30200080B
:10014000E3020008E3020008E3020008E3020008FB
:10015000E3020008E3020008E3020008E3020008EB
:10016000E3020008E3020008E3020008E3020008DB
:10017000E3020008A5340008E3020008E3020008D7
:10018000E3020008E3020008C1400008E30200089F
:10019000E3020008E3020008E3020008E3020008AB
:1001A000E3020008E3020008E3020008E30200089B
:1001B000E3020008E3020008E3020008E30200088B
:1001C000E3020008E3020008E3020008E30200087B
:1001D000E302000891340008E3020008E30200088B
:1001E000E3020008E3020008E3020008E30200085B
:1001F000E3020008E3020008E3020008E30200084B
:10020000E3020008E3020008E3020008E30200083A
:10021000E3020008E3020008E3020008E30200082A
:10022000E3020008E3020008E3020008E30200081A
:10023000E3020008E3020008E3020008E30200080A
:10024000E3020008E3020008E3020008E3020008FA
:10025000E3020008E3020008E3020008E3020008EA
:10026000E3020008E3020008E3020008E3020008DA
:10027000E3020008E3020008E3020008E3020008CA
:10028000E3020008E3020008E3020008E3020008BA
:10029000E3020008E3020008E3020008E3020008AA
:1002A000E3020008E3020008E3020008E30200089A
:1002B000E3020008E3020008E3020008E30200088A
:1002C000E3020008E3020008E3020008E30200087A
:1002D000E3020008E3020008E3020008E30200086A
:1002E00002E000F000F8FEE772B6374880F30888B5
:1002F000364880F3098836483649086040F20000E5
:10030000CCF200004EF63471CEF200010860BFF36B
:100310004F8FBFF36F8F40F20000C0F2F0004EF637
:100320008851CEF200010860BFF34F8FBFF36F8F8B
:100330004FF00000E1EE100A4EF63C71CEF20001E3
:100340000860062080F31488BFF36F8F02F016FB5D
:1003500003F03AFB4FF055301F491B4A91423CBF16
:1003600041F8040BFAE71D49184A91423CBF41F895
:10037000040BFAE71A491B4A1B4B9A423EBF51F83D
:10038000040B42F8040BF8E700201849184A914280
:100390003CBF41F8040BFAE702F02EFB03F098FB98
:1003A000144C154DAC4203DA54F8041B8847F9E7A6
:1003B00000F042F8114C124DAC4203DA54F8041B21
:1003C0008847F9E702F016BB000600200022002053
:1003D0000000000808ED00E00000002000060020FA
:1003E000004500080022002064220020682200202E
:1003F000C4470020E0020008E0020008E002000814
:10040000E00200082DE9F04F2DED108AC1F80CD064
:10041000D0F80CD0BDEC108ABDE8F08F002383F338
:1004200011882846A047002001F02CFEFEE701F0CD
:10043000BBFD00DFFEE7000038B500F0DBFB02F09B
:100440005DFA054602F090FA0446D0B90F4B9D4282
:1004500019D001339D4241F2883512BF0446002570
:100460000124002002F054FA0CB100F077F800F0FB
:1004700097FD00F03BFC284600F01EF900F06EF8F6
:10048000F9E70025EDE70546EBE700BF010007B0FF
:1004900008B500F0F7FBA0F120035842584108BD11
:1004A00007B541F21203022101A8ADF8043000F0B3
:1004B00007FC03B05DF804FB38B5302383F31188E3
:1004C000174803680BB101F0A9FE0023154A4FF449
:1004D0007A71134801F098FE002383F31188124CBF
:1004E000236813B12368013B2360636813B1636819
:1004F000013B63600D4D2B7833B963687BB90220F3
:1005000000F0BEFC322363602B78032B07D16368B5
:100510002BB9022000F0B4FC4FF47A73636038BD4D
:1005200068220020B90400088823002080220020CF
:10053000084B187003280CD8DFE800F00805020803
:10054000022000F08DBC022000F078BC024B00229B
:100550005A6070478022002088230020F8B5504B55
:10056000504A1C461968013100F0998004339342C7
:10057000F8D162684C4B9A4240F291804B4B9B6899
:1005800003F1006303F500339A4280F08880002075
:1005900000F0C6FB0220FFF7CBFF454B0021D3F84C
:1005A000E820C3F8E810D3F81021C3F81011D3F8ED
:1005B0001021D3F8EC20C3F8EC10D3F81421C3F8C1
:1005C0001411D3F81421D3F8F020C3F8F010D3F8A5
:1005D0001821C3F81811D3F81821D3F8802042F05D
:1005E0000062C3F88020D3F8802022F00062C3F8B4
:1005F0008020D3F88020D3F8802042F00072C3F826
:100600008020D3F8802022F00072C3F88020D3F835
:10061000803072B64FF0E023C3F8084DD4E90004EF
:10062000BFF34F8FBFF36F8F224AC2F88410BFF31E
:100630004F8F536923F480335361BFF34F8FD2F848
:10064000803043F6E076C3F3C905C3F34E335B0154
:1006500003EA060C29464CEA81770139C2F8747224
:10066000F9D2203B13F1200FF2D1BFF34F8FBFF32C
:100670006F8FBFF34F8FBFF36F8F536923F4003336
:1006800053610023C2F85032BFF34F8FBFF36F8F17
:10069000302383F31188854680F308882047F8BD0E
:1006A0000000020820000208FFFF010800220020CD
:1006B0000044025800ED00E02DE9F04F93B0B44B38
:1006C0002022FF2100900AA89D6800F013FCB14A87
:1006D0001378A3B90121B04811700360302383F36C
:1006E000118803680BB101F099FD0023AB4A4FF468
:1006F0007A71A94801F088FD002383F31188009BDB
:1007000013B1A74B009A1A60A64A1378032B03D0A3
:1007100000231370A24A53604FF0000A009CD34696
:100720005646D146012000F09BFB24B19C4B1B6830
:10073000002B00F02682002000F0A4FA0390039B17
:10074000002BF2DB012000F079FB039B213B1F2BE8
:10075000E8D801A252F823F0D907000801080008E0
:100760009508000825070008250700082507000848
:1007700027090008F70A0008110A0008730A000890
:100780009B0A0008C10A000825070008D30A0008D0
:1007900025070008450B0008790800082507000810
:1007A000890B0008E50700087908000825070008FC
:1007B000730A000825070008250700082507000818
:1007C0002507000825070008250700082507000859
:1007D00025070008950800080220FFF759FE0028A9
:1007E00040F0F981009B022105A8BAF1000F08BF73
:1007F0001C4641F21233ADF8143000F061FA91E773
:100800004FF47A7000F03EFA071EEBDB0220FFF790
:100810003FFE0028E6D0013F052F00F2DE81DFE831
:1008200007F0030A0D1013360523042105A80593CC
:1008300000F046FA17E004215548F9E704215A4828
:10084000F6E704215948F3E74FF01C08404608F149
:10085000040800F067FA0421059005A800F030FABA
:10086000B8F12C0FF2D101204FF0000900FA07F780
:1008700047EA0B0B5FFA8BFB00F088FB26B10BF00D
:100880000B030B2B08BF0024FFF70AFE4AE70421E5
:100890004748CDE7002EA5D00BF00B030B2BA1D1C1
:1008A0000220FFF7F5FD074600289BD00120002617
:1008B00000F036FA0220FFF73BFE1FFA86F84046AA
:1008C00000F03EFA0446B0B1039940460136A1F16A
:1008D00040025142514100F043FA0028EDD1BA469E
:1008E000044641F21213022105A83E46ADF8143029
:1008F00000F0E6F916E725460120FFF719FE244B24
:100900009B68AB4207D9284600F00CFA013040F052
:1009100067810435F3E70025224BBA463E461D7039
:100920001F4B5D60A8E7002E3FF45CAF0BF00B039C
:100930000B2B7FF457AF0220FFF7FAFD322000F0B7
:10094000A1F9B0F10008FFF64DAF18F003077FF4EE
:1009500049AF0F4A08EB0503926893423FF642AF56
:10096000B8F5807F3FF73EAF124BB845019323DDCA
:100970004FF47A7000F086F90390039A002AFFF68C
:1009800031AF039A0137019B03F8012BEDE700BF5C
:10099000002200208423002068220020B9040008DF
:1009A000882300208022002004220020082200202A
:1009B0000C22002084220020C820FFF769FD074692
:1009C00000283FF40FAF1F2D11D8C5F120020AAB4C
:1009D00025F0030084494245184428BF424601924D
:1009E00000F062FA019AFF217F4800F083FA4FEA93
:1009F000A803C8F387027C492846019300F082FAD5
:100A0000064600283FF46DAF019B05EB830533E7F5
:100A10000220FFF73DFD00283FF4E4AE00F0BEF9F0
:100A200000283FF4DFAE0027B846704B9B68BB42FE
:100A300018D91F2F11D80A9B01330ED027F00303BA
:100A400012AA134453F8203C05934046042205A9FA
:100A5000043700F007FB8046E7E7384600F062F90C
:100A60000590F2E7CDF81480042105A800F028F9DC
:100A700002E70023642104A8049300F017F900287A
:100A80007FF4B0AE0220FFF703FD00283FF4AAAECA
:100A9000049800F079F90590E6E70023642104A8A2
:100AA000049300F003F900287FF49CAE0220FFF7C6
:100AB000EFFC00283FF496AE049800F067F9EAE7EF
:100AC0000220FFF7E5FC00283FF48CAE00F076F939
:100AD000E1E70220FFF7DCFC00283FF483AE05A924
:100AE000142000F071F907460421049004A800F0D6
:100AF000E7F83946B9E7322000F0C4F8071EFFF6E0
:100B000071AEBB077FF46EAE384A07EB09039268FB
:100B100093423FF667AE0220FFF7BAFC00283FF48D
:100B200061AE27F003074F44B9453FF4A5AE4846F0
:100B300009F1040900F0F6F80421059005A800F079
:100B4000BFF8F1E74FF47A70FFF7A2FC00283FF4FA
:100B500049AE00F023F9002844D00A9B01330BD0A2
:100B600008220AA9002000F0CDF900283AD020225E
:100B7000FF210AA800F0BEF9FFF792FC1C4801F023
:100B800087FA13B0BDE8F08F002E3FF42BAE0BF0C8
:100B90000B030B2B7FF426AE0023642105A80593DD
:100BA00000F084F8074600287FF41CAE0220FFF70F
:100BB0006FFC804600283FF415AEFFF771FC41F250
:100BC000883001F065FA059800F02AFA46463C465E
:100BD00000F0DCF9A6E506464EE64FF0000901E616
:100BE000BA467EE637467CE68422002000220020BA
:100BF000A0860100704700002DE9F84F4FF47A738A
:100C000006460D46002402FB03F7DFF85080DFF8AC
:100C1000509098F900305FFA84FA5A1C01D0A34230
:100C200012D159F824002A4631460368D3F820B07F
:100C30003B46D847854207D1074B012083F800A0E7
:100C4000BDE8F88F0124E4E7002CFBD04FF4FA70E4
:100C500001F01EFA0020F3E7D42300201022002028
:100C60001422002070B504464FF47A76412C2546B4
:100C700028BF412506FB05F001F00AFA641BF5D1F7
:100C800070BD0000002307B5024601210DF10700E9
:100C90008DF80730FFF7B0FF20B19DF8070003B0D3
:100CA0005DF804FB4FF0FF30F9E700000A4604212D
:100CB00008B5FFF7A1FF80F00100C0B2404208BDB7
:100CC000074B0A4630B41978064B53F821400146C9
:100CD00023682046DD69044BAC4630BC604700BF4A
:100CE000D423002014220020A086010070B50A4EF3
:100CF00000240A4D01F0EAFC3080286833888342E2
:100D000008D901F0DFFC2B6804440133B4F5003F3F
:100D10002B60F2D370BD00BFD623002090230020AB
:100D200001F0A2BD00F1006000F5003000687047DE
:100D300000F10060920000F5003001F023BD0000DA
:100D4000054B1A68054B1B889B1A834202D9104435
:100D500001F0B8BC0020704790230020D62300206B
:100D600038B50446074D29B128682044BDE838400D
:100D700001F0C0BC2868204401F0AAFC0028F3D090
:100D800038BD00BF902300200020704700F1FF50C5
:100D900000F58F10D0F8000870470000064991F860
:100DA000243033B100230822086A81F82430FFF789
:100DB000BFBF0120704700BF94230020014B18687B
:100DC000704700BF0010005C194B01380322084433
:100DD00070B51D68174BC5F30B042D0C1E88A64279
:100DE0000BD15C680A46013C824213460FD214F9CB
:100DF000016F4EB102F8016BF6E7013A03F1080307
:100E0000ECD181420B4602D22C2203F8012B0424A0
:100E1000094A1688AE4204D1984284BF967803F8F6
:100E2000016B013C02F10402F3D1581A70BD00BFFE
:100E30000010005C1C220020D8410008022804D1C8
:100E4000054B4FF080629A6170470128FCD1034B3B
:100E50004FF48032F7E700BF000C02580018025828
:100E6000022804D1044B4FF480629A617047012834
:100E700001D1024B98617047000C025800180258CB
:100E8000022805D1064A536983F480635361704791
:100E90000128FCD1034A536983F00103F6E700BF40
:100EA000000C025800180258002310B5934203D0DA
:100EB000CC5CC4540133F9E710BD0000013810B513
:100EC00010F9013F3BB191F900409C4203D11AB1A6
:100ED0000131013AF4E71AB191F90020981A10BDD6
:100EE0001046FCE703460246D01A12F9011B0029FE
:100EF000FAD1704702440346934202D003F8011B23
:100F0000FAE770472DE9F8431F4D14460746884617
:100F100095F8242052BBDFF870909CB395F82430EC
:100F20002BB92022FF2148462F62FFF7E3FF95F8F7
:100F300024004146C0F1080205EB8000A24228BF10
:100F40002246D6B29200FFF7AFFF95F82430A41BDB
:100F500017441E449044E4B2F6B2082E85F824608B
:100F6000DBD1FFF71BFF0028D7D108E02B6A03EB8A
:100F700082038342CFD0FFF711FF0028CBD100209E
:100F8000BDE8F8830120FBE794230020024B1A7888
:100F9000024B1A70704700BFD4230020102200209B
:100FA00038B51A4C1A4D204600F0C6FB294620469B
:100FB00000F0EEFB2D684FF47A70D5F89020D2F84F
:100FC000043843F00203C2F80438FFF74BFE11491E
:100FD000284600F0EBFCD5F890200F4DD2F80438ED
:100FE000286823F002030D49A042C2F804384FF4E8
:100FF000E1330B6001D000F0FDFA6868A04204D034
:101000000649BDE8384000F0F5BA38BDB82A0020DE
:10101000D4420008DC42000814220020BC23002037
:101020000C4B70B50C4D04461E780C4B55F8262021
:101030009A420DD00A4B002118221846FFF75AFF9A
:101040000460014655F82600BDE8704000F0D2BAB1
:1010500070BD00BFD423002014220020B82A002035
:10106000BC23002030B50A44084D91420DD011F840
:10107000013B5840082340F30004013B2C4013F08F
:10108000FF0384EA5000F6D1EFE730BD2083B8EDCE
:10109000026843681143016003B1184770470000BC
:1010A000024A136843F0C0031360704700780040A1
:1010B00013B50E4C204600F091FA04F11400002301
:1010C0004FF400720A49009400F04EF9094B4FF4B6
:1010D0000072094904F13800009400F0C7F9074A8A
:1010E000074BC4E9172302B010BD00BFD82300206E
:1010F00044240020A110000844260020007800406D
:1011000000E1F505037C30B5244C002918BF0C46DE
:10111000012B11D1224B98420ED1224BD3F8E8205B
:1011200042F08042C3F8E820D3F8102142F0804218
:10113000C3F81021D3F810312268036EC16D03EBA0
:1011400052038466B3FBF2F36268150442BF23F0D6
:10115000070503F0070343EA4503CB60A36843F0A8
:1011600040034B60E36843F001038B6042F49673E5
:1011700043F001030B604FF0FF330B62510505D5BF
:1011800012F0102205D0B2F1805F04D080F86430F4
:1011900030BD7F23FAE73F23F8E700BFE8410008AE
:1011A000D8230020004402582DE9F047C66D0546BB
:1011B0003768F469210734621AD014F0080118BFA7
:1011C0004FF48071E20748BF41F02001A3074FF0C0
:1011D000300348BF41F04001600748BF41F0800143
:1011E00083F31188281DFFF753FF002383F3118831
:1011F000E2050AD5302383F311884FF48061281D5E
:10120000FFF746FF002383F311884FF030094FF0BA
:10121000000A14F0200838D13B0616D54FF03009EB
:1012200005F1380A200610D589F31188504600F0E0
:1012300051F9002836DA0821281DFFF729FF27F089
:1012400080033360002383F31188790614D5620686
:1012500012D5302383F31188D5E913239A4208D19C
:101260002B6C33B127F040071021281DFFF710FF2A
:101270003760002383F31188E30618D5AA6E13693B
:10128000ABB15069BDE8F047184789F31188736A1C
:10129000284695F86410194000F0BAF98AF31188CD
:1012A000F469B6E7B06288F31188F469BAE7BDE87B
:1012B000F0870000F8B51546826804460B46AA423E
:1012C00000D28568A1692669761AB5420BD2184604
:1012D0002A46FFF7E9FDA3692B44A3612846A368CA
:1012E0005B1BA360F8BD0CD9AF1B18463246FFF755
:1012F000DBFD3A46E1683044FFF7D6FDE3683B4446
:10130000EBE718462A46FFF7CFFDE368E5E7000064
:1013100083689342F7B50446154600D28568D4E940
:101320000460361AB5420BD22A46FFF7BDFD636949
:101330002B4463612846A3685B1BA36003B0F0BD28
:101340000DD93246AF1B0191FFF7AEFD01993A4628
:10135000E0683144FFF7A8FDE3683B44E9E72A462B
:10136000FFF7A2FDE368E4E710B50A440024C36177
:10137000029B8460C16002610362C0E90000C0E9B1
:10138000051110BD08B5D0E90532934201D182683C
:1013900082B98268013282605A1C42611970002150
:1013A000D0E904329A4224BFC368436100F08CFE46
:1013B000002008BD4FF0FF30FBE7000070B5302380
:1013C00004460E4683F31188A568A5B1A368A269F7
:1013D000013BA360531CA36115782269934224BF8B
:1013E000E368A361E3690BB120469847002383F3C8
:1013F0001188284607E03146204600F055FE0028B7
:10140000E2DA85F3118870BD2DE9F74F04460E46E8
:1014100017469846D0F81C904FF0300A8AF311888E
:101420004FF0000B154665B12A4631462046FFF7BE
:1014300041FF034660B94146204600F035FE0028D2
:10144000F1D0002383F31188781B03B0BDE8F08F3F
:10145000B9F1000F03D001902046C847019B8BF3E0
:101460001188ED1A1E448AF31188DCE7C160C3615C
:10147000009B82600362C0E905111144C0E90000CD
:1014800001617047F8B504460D461646302383F3D4
:101490001188A768A7B1A368013BA36063695A1CC0
:1014A00062611D70D4E904329A4224BFE36863612B
:1014B000E3690BB120469847002080F3118807E0CC
:1014C0003146204600F0F0FD0028E2DA87F311886B
:1014D000F8BD0000D0E9052310B59A4201D1826819
:1014E0007AB982680021013282605A1C82611C78BC
:1014F00003699A4224BFC368836100F0E5FD20467A
:1015000010BD4FF0FF30FBE72DE9F74F04460E46C4
:1015100017469846D0F81C904FF0300A8AF311888D
:101520004FF0000B154665B12A4631462046FFF7BD
:10153000EFFE034660B94146204600F0B5FD0028A5
:10154000F1D0002383F31188781B03B0BDE8F08F3E
:10155000B9F1000F03D001902046C847019B8BF3DF
:101560001188ED1A1E448AF31188DCE7026843688B
:101570001143016003B11847704700001430FFF7B2
:1015800043BF00004FF0FF331430FFF73DBF0000B2
:101590003830FFF7B9BF00004FF0FF333830FFF7A6
:1015A000B3BF00001430FFF709BF00004FF0FF3158
:1015B0001430FFF703BF00003830FFF763BF0000AF
:1015C0004FF0FF323830FFF75DBF0000012914BF34
:1015D0006FF0130000207047FFF76ABD044B0360F3
:1015E00000234360C0E9023301230374704700BF46
:1015F0000042000810B53023044683F31188FFF73A
:1016000081FD02230020237480F3118810BD0000A7
:1016100038B5C36904460D461BB904210844FFF7D9
:10162000A5FF294604F11400FFF7ACFE002806DAF6
:10163000201D4FF40061BDE83840FFF797BF38BD6B
:10164000026843681143016003B118477047000006
:1016500013B5406B00F58054D4F8A4381A6811789B
:10166000042914D1017C022911D11979012312898D
:101670008B4013420BD101A94C3002F05BF8D4F837
:10168000A4480246019B2179206800F0DFF902B0EE
:1016900010BD0000143001F0DDBF00004FF0FF333B
:1016A000143001F0D7BF00004C3002F0AFB800009A
:1016B0004FF0FF334C3002F0A9B80000143001F0B5
:1016C000ABBF00004FF0FF31143001F0A5BF0000A8
:1016D0004C3002F07BB800004FF0FF324C3002F08B
:1016E00075B800000020704710B500F58054D4F89C
:1016F000A4381A681178042917D1017C022914D161
:101700005979012352898B4013420ED1143001F0D4
:101710003DFF024648B1D4F8A4484FF440736179C4
:101720002068BDE8104000F07FB910BD406BFFF7A6
:10173000DBBF0000704700007FB5124B0125042677
:10174000044603600023057400F1840243602946C7
:10175000C0E902330C4B0290143001934FF44073F4
:10176000009601F0EFFE094B04F69442294604F17D
:101770004C000294CDE900634FF4407301F0B6FFD2
:1017800004B070BD284200082D170008511600084B
:101790000A68302383F311880B790B3342F8230056
:1017A0004B79133342F823008B7913B10B3342F892
:1017B000230000F58053C3F8A4180223037400200B
:1017C00080F311887047000038B5037F044613B1D9
:1017D00090F85430ABB90125201D0221FFF730FFEE
:1017E00004F114006FF00101257700F079FC04F199
:1017F0004C0084F854506FF00101BDE8384000F00F
:101800006FBC38BD10B5012104460430FFF718FF46
:101810000023237784F8543010BD000038B5044607
:101820000025143001F0A6FE04F14C00257701F0EC
:1018300075FF201D84F854500121FFF701FF204659
:10184000BDE83840FFF750BF90F8803003F06003E8
:10185000202B06D190F881200023212A03D81F2AAB
:1018600006D800207047222AFBD1C0E91D3303E0CF
:10187000034A426707228267C3670120704700BF9F
:101880003422002037B500F58055D5F8A4381A6801
:10189000117804291AD1017C022917D11979012361
:1018A00012898B40134211D100F14C04204601F003
:1018B000F5FF58B101A9204601F03CFFD5F8A44836
:1018C0000246019B2179206800F0C0F803B030BDCA
:1018D00001F10B03F0B550F8236085B004460D46C6
:1018E000FEB1302383F3118804EB8507301D0821F6
:1018F000FFF7A6FEFB6806F14C005B691B681BB195
:10190000019001F025FF019803A901F013FF0246A1
:1019100048B1039B2946204600F098F8002383F342
:10192000118805B0F0BDFB685A691268002AF5D02D
:101930001B8A013B1340F1D104F18002EAE7000069
:10194000133138B550F82140ECB1302383F31188BE
:1019500004F58053D3F8A4281368527903EB82036B
:10196000DB689B695D6845B104216018FFF768FE7C
:10197000294604F1140001F013FE2046FFF7B4FEDF
:10198000002383F3118838BD7047000001F0CAB806
:1019900001234022002110B5044600F8303BFFF738
:1019A000A9FA0023C4E9013310BD000010B53023AB
:1019B000044683F311882422416000210C30FFF794
:1019C00099FA204601F0D0F802230020237080F31A
:1019D000118810BD70B500EB8103054650690E46B5
:1019E0001446DA6018B110220021FFF783FAA069CB
:1019F00018B110220021FFF77DFA31462846BDE8D4
:101A0000704001F0B7B9000083682022002103F084
:101A1000011310B5044683601030FFF76BFA2046BF
:101A2000BDE8104001F032BAF0B4012500EB8104AA
:101A300047898D40E4683D43A469458123600023C4
:101A4000A2606360F0BC01F04FBA0000F0B4012561
:101A500000EB810407898D40E4683D43646905819A
:101A600023600023A2606360F0BC01F0C5BA0000EF
:101A700070B5022300250446242203702946C0F8CD
:101A800088500C3040F8045CFFF734FA204684F8A4
:101A9000705001F003F963681B6823B129462046A2
:101AA000BDE87040184770BD0378052B10B504469B
:101AB0000AD080F88C300523037043681B680BB193
:101AC000042198470023A36010BD00000178052978
:101AD00006D190F88C20436802701B6803B1184748
:101AE0007047000070B590F87030044613B10023C1
:101AF00080F8703004F18002204601F0EBF9636851
:101B00009B68B3B994F8803013F0600535D000219C
:101B1000204601F0DDFC0021204601F0CDFC636889
:101B20001B6813B1062120469847062384F87030BD
:101B300070BD204698470028E4D0B4F88630A26FE4
:101B40009A4288BFA36794F98030A56F002B4FF0AD
:101B5000300380F20381002D00F0F280092284F826
:101B6000702083F3118800212046D4E91D23FFF75C
:101B70006DFF002383F31188DAE794F8812003F0E6
:101B80007F0343EA022340F20232934200F0C58011
:101B900021D8B3F5807F48D00DD8012B3FD0022B40
:101BA00000F09380002BB2D104F188026267022218
:101BB000A267E367C1E7B3F5817F00F09B80B3F5CF
:101BC000407FA4D194F88230012BA0D1B4F88830A2
:101BD00043F0020332E0B3F5006F4DD017D8B3F5F0
:101BE000A06F31D0A3F5C063012B90D86368204665
:101BF00094F882205E6894F88310B4F88430B0477B
:101C0000002884D0436863670368A3671AE0B3F5CC
:101C1000106F36D040F6024293427FF478AF5C4BAF
:101C200063670223A3670023C3E794F88230012B84
:101C30007FF46DAFB4F8883023F00203A4F8883045
:101C4000C4E91D55E56778E7B4F88030B3F5A06FB7
:101C50000ED194F88230204684F88A3001F07CF866
:101C600063681B6813B10121204698470323237042
:101C70000023C4E91D339CE704F18B036367012350
:101C8000C3E72378042B10D1302383F31188204637
:101C9000FFF7BAFE85F311880321636884F88B503F
:101CA00021701B680BB12046984794F88230002BB6
:101CB000DED084F88B300423237063681B68002B0C
:101CC000D6D0022120469847D2E794F884302046A7
:101CD0001D0603F00F010AD501F0EEF8012804D02B
:101CE00002287FF414AF2B4B9AE72B4B98E701F0B7
:101CF000D5F8F3E794F88230002B7FF408AF94F81E
:101D0000843013F00F01B3D01A06204602D501F03B
:101D1000F7FBADE701F0E8FBAAE794F88230002B6F
:101D20007FF4F5AE94F8843013F00F01A0D01B06B9
:101D3000204602D501F0CCFB9AE701F0BDFB97E706
:101D4000142284F8702083F311882B462A462946F2
:101D50002046FFF769FE85F31188E9E65DB115229B
:101D600084F8702083F3118800212046D4E91D23D4
:101D7000FFF75AFEFDE60B2284F8702083F31188EA
:101D80002B462A4629462046FFF760FEE3E700BFC0
:101D900058420008504200085442000838B590F8F4
:101DA00070300446002B3ED0063BDAB20F2A34D8FE
:101DB0000F2B32D8DFE803F03731310822323131CE
:101DC0003131313131313737856FB0F886309D424E
:101DD00014D2C3681B8AB5FBF3F203FB12556DB92D
:101DE000302383F311882B462A462946FFF72EFE1F
:101DF00085F311880A2384F870300EE0142384F8E8
:101E00007030302383F31188002320461A46194688
:101E1000FFF70AFE002383F3118838BDC36F03B1B7
:101E200098470023E7E70021204601F051FB0021FD
:101E3000204601F041FB63681B6813B10621204670
:101E400098470623D7E7000010B590F87030044695
:101E5000142B29D017D8062B05D001D81BB110BDE3
:101E6000093B022BFBD80021204601F031FB002169
:101E7000204601F021FB63681B6813B10621204650
:101E80009847062319E0152BE9D10B2380F8703011
:101E9000302383F3118800231A461946FFF7D6FD35
:101EA000002383F31188DAE7C3689B695B68002B22
:101EB000D5D1C36F03B19847002384F87030CEE7C3
:101EC00000238268037503691B6899689142FBD2FD
:101ED0005A6803604260106058607047002382684F
:101EE000037503691B6899689142FBD85A680360BF
:101EF000426010605860704708B50846302383F38D
:101F000011880B7D032B05D0042B0DD02BB983F347
:101F1000118808BD8B6900221A604FF0FF3383617E
:101F2000FFF7CEFF0023F2E7D1E9003213605A60D9
:101F3000F3E70000FFF7C4BF054BD96808751868C0
:101F4000026853601A600122D8600275FEF75ABA1F
:101F5000482800200C4B30B5DD684B1C87B0044688
:101F60000FD02B46094A684600F04EF92046FFF78D
:101F7000E3FF009B13B1684600F050F9A86907B071
:101F800030BDFFF7D9FFF9E748280020F91E000807
:101F9000044B1A68DB6890689B68984294BF0020E5
:101FA0000120704748280020084B10B51C68D868ED
:101FB000226853601A600122DC602275FFF78EFFF1
:101FC00001462046BDE81040FEF71CBA4828002014
:101FD00038B5074C01230025064907482370656082
:101FE00001F09AFC0223237085F3118838BD00BFED
:101FF000B02A0020604200084828002000F044B9C0
:10200000034A516853685B1A9842FBD8704700BF77
:10201000001000E08B600223086108468B82704745
:102020008368A3F1840243F8142C026943F8442C1A
:10203000426943F8402C094A43F8242CC268A3F1B2
:10204000200043F8182C022203F80C2C002203F87D
:102050000B2C034A43F8102C704700BF1D040008E6
:102060004828002008B5FFF7DBFFBDE80840FFF770
:1020700061BF0000024BDB6898610F20FFF75CBF77
:1020800048280020302383F31188FFF7F3BF0000B6
:1020900008B50146302383F311880820FFF75AFF63
:1020A000002383F3118808BD064BDB6839B1426811
:1020B00018605A60136043600420FFF74BBF4FF075
:1020C000FF307047482800200368984206D01A68FD
:1020D0000260506018469961FFF72CBF70470000FE
:1020E00038B504460D462068844200D138BD0368E7
:1020F00023605C608561FFF71DFFF4E7036810B59E
:102100009C68A2420CD85C688A600B604C602160BD
:10211000596099688A1A9A604FF0FF33836010BD46
:10212000121B1B68ECE700000A2938BF0A2170B5B2
:1021300004460D460A26601901F0E6FB01F0CEFBCD
:10214000041BA54203D8751C04462E46F3E70A2E4D
:1021500004D90120BDE8704001F01EBC70BD000034
:10216000F8B5144B0D460A2A4FF00A07D96103F15E
:102170001001826038BF0A2241601969144601606B
:1021800048601861A81801F0AFFB01F0A7FB431BE2
:102190000646A34206D37C1C28192746354601F083
:1021A000B3FBF2E70A2F04D90120BDE8F84001F0A3
:1021B000F3BBF8BD48280020F8B506460D4601F0EF
:1021C0008DFB0F4A134653F8107F9F4206D12A46D3
:1021D00001463046BDE8F840FFF7C2BFD169BB6891
:1021E000441A2C1928BF2C46A34202D92946FFF7CE
:1021F0009BFF224631460348BDE8F840FFF77EBF0B
:102200004828002058280020C0E90323002310B4E8
:102210005DF8044B4361FFF7CFBF000010B5194CC8
:10222000236998420DD08168D0E9003213605A606A
:102230009A680A449A60002303604FF0FF33A36159
:1022400010BD0268234643F8102F5360002202603D
:1022500022699A4203D1BDE8104001F04FBB936858
:1022600081680B44936001F039FB2269E16992684F
:10227000441AA242E4D91144BDE81040091AFFF7FC
:1022800053BF00BF482800202DE9F047DFF8BC808D
:1022900008F110072C4ED8F8105001F01FFBD8F8A9
:1022A0001C40AA68031B9A423ED814444FF0000910
:1022B000D5E90032C8F81C4013605A60C5F8009098
:1022C000D8F81030B34201D101F018FB89F311881E
:1022D000D5E9033128469847302383F311886B6989
:1022E000002BD8D001F0FAFA6A69A0EB0409824603
:1022F0004A450DD2022001F04FFB0022D8F81030E1
:10230000B34208D151462846BDE8F047FFF728BF41
:10231000121A2244F2E712EB09092946384638BF5F
:102320004A46FFF7EBFEB5E7D8F81030B34208D0C5
:102330001444C8F81C00211AA960BDE8F047FFF753
:10234000F3BEBDE8F08700BF5828002048280020D1
:1023500000207047FEE70000704700004FF0FF309C
:102360007047000002290CD0032904D00129074836
:1023700018BF00207047032A05D8054800EBC200AB
:102380007047044870470020704700BF384300087A
:1023900044220020EC42000870B59AB00546084679
:1023A000144601A900F0C2F801A8FEF79BFD431CEA
:1023B0000022C6B25B001046C5E900342370032337
:1023C000023404F8013C01ABD1B202348E4201D890
:1023D0001AB070BD13F8011B013204F8010C04F8A7
:1023E000021CF1E708B5302383F311880348FFF797
:1023F00049FA002383F3118808BD00BFB82A0020E2
:1024000090F8803003F01F02012A07D190F8812054
:102410000B2A03D10023C0E91D3315E003F060034C
:10242000202B08D1B0F884302BB990F88120212AD4
:1024300003D81F2A04D8FFF707BA222AEBD0FAE7FD
:10244000034A426707228267C3670120704700BFC3
:102450003B22002007B5052917D8DFE801F019163F
:1024600003191920302383F31188104A01210190A8
:10247000FFF7B0FA019802210D4AFFF7ABFA0D48B9
:10248000FFF7CCF9002383F3118803B05DF804FB58
:10249000302383F311880748FFF796F9F2E73023DA
:1024A00083F311880348FFF7ADF9EBE78C4200088E
:1024B000B0420008B82A002038B50C4D0C4C2A4612
:1024C0000C4904F10800FFF767FF05F1CA0204F1A7
:1024D00010000949FFF760FF05F5CA7204F1180002
:1024E0000649BDE83840FFF757BF00BF90430020C2
:1024F000442200206C420008764200088142000815
:1025000070B5044608460D46FEF7ECFCC6B2204600
:10251000013403780BB9184670BD32462946FEF7E0
:10252000CDFC0028F3D10120F6E700002DE9F047AB
:1025300005460C46FEF7D6FC2C49C6B22846FFF7E6
:10254000DFFF08B10836F6B229492846FFF7D8FF61
:1025500008B11036F6B2632E0BD8DFF89080DFF8A2
:102560009090244FDFF898A02E7846B92670BDE8E9
:10257000F08729462046BDE8F04701F00FBE252E22
:1025800030D1072241462846FEF798FC80B91A4B05
:10259000224603F10C0153F8040B8B4242F8040B62
:1025A000F9D1198807359B780F3411809370DBE7D8
:1025B000082249462846FEF781FC98B9A21C0F4B19
:1025C000197802320909C95D02F8041C13F8011BCD
:1025D00001F00F015345C95D02F8031CF0D1183416
:1025E0000835C1E7013504F8016BBDE75843000821
:1025F00081420008704300086043000800E8F11FB2
:102600000CE8F11FBFF34F8F044B1A695107FCD13F
:10261000D3F810215207F8D1704700BF00200052B4
:1026200008B50D4B1B78ABB9FFF7ECFF0B4BDA6825
:10263000D10704D50A4A5A6002F188325A60D3F8A9
:102640000C21D20706D5064AC3F8042102F18832CC
:10265000C3F8042108BD00BFEE4500200020005251
:102660002301674508B5114B1B78F3B9104B1A6964
:10267000510703D5DA6842F04002DA60D3F810213E
:10268000520705D5D3F80C2142F04002C3F80C21C3
:10269000FFF7B8FF064BDA6842F00102DA60D3F8C0
:1026A0000C2142F00102C3F80C2108BDEE450020C8
:1026B000002000520F289ABF00F5806040040020DF
:1026C000704700004FF40030704700001020704742
:1026D0000F2808B50BD8FFF7EDFF00F500330268AF
:1026E000013204D104308342F9D1012008BD002019
:1026F000FCE700000F2838B505463FD8FFF782FFFA
:102700001F4CFFF78DFF4FF0FF3307286361C4F8BC
:1027100014311DD82361FFF775FF030243F0240332
:10272000E360E36843F08003E36023695A07FCD465
:102730002846FFF767FFFFF7BDFF4FF4003100F0B9
:10274000F5F82846FFF78EFFBDE83840FFF7C0BF19
:10275000C4F81031FFF756FFA0F108031B0243F045
:102760002403C4F80C31D4F80C3143F08003C4F8CE
:102770000C31D4F810315B07FBD4D9E7002038BD09
:10278000002000522DE9F84F05460C46104645EA58
:102790000203DE0602D00020BDE8F88F20F01F0003
:1027A000DFF8BCB0DFF8BCA0FFF73AFF04EB00088D
:1027B000444503D10120FFF755FFEDE720222946CC
:1027C000204601F0DBFC10B920352034F0E72B4621
:1027D00005F120021F68791CDDD104339A42F9D13A
:1027E00005F178431B481C4EB3F5801F1B4B38BFC7
:1027F000184603F1F80332BFD946D1461E46FFF70B
:1028000001FF0760A5EB040C336804F11C0143F0E1
:1028100002033360231FD9F8007017F00507FAD1BF
:1028200053F8042F8B424CF80320F4D1BFF34F8FA1
:10283000FFF7E8FE4FF0FF332022214603602846D1
:10284000336823F00203336001F098FC0028BBD00A
:102850003846B0E7142100520C20005214200052D8
:10286000102000521021005210B5084C237828B1D6
:102870001BB9FFF7D5FE0123237010BD002BFCD040
:102880002070BDE81040FFF7EDBE00BFEE45002010
:102890000244074BD2B210B5904200D110BD441C87
:1028A00000B253F8200041F8040BE0B2F4E700BF97
:1028B000504000580E4B30B51C6F240405D41C6FDB
:1028C0001C671C6F44F400441C670A4C02442368D4
:1028D000D2B243F480732360074B904200D130BDE5
:1028E000441C51F8045B00B243F82050E0B2F4E716
:1028F00000440258004802585040005807B50122D1
:1029000001A90020FFF7C4FF019803B05DF804FBA4
:1029100013B50446FFF7F2FFA04205D0012201A93A
:1029200000200194FFF7C6FF02B010BD0144BFF3C1
:102930004F8F064B884204D3BFF34F8FBFF36F8F87
:102940007047C3F85C022030F4E700BF00ED00E000
:10295000034B1A681AB9034AD2F8D0241A60704798
:10296000F04500200040025808B5FFF7F1FF024B88
:102970001868C0F3806008BDF045002070B5BFF353
:102980004F8FBFF36F8F1A4A0021C2F85012BFF366
:102990004F8FBFF36F8F536943F400335361BFF31D
:1029A0004F8FBFF36F8FC2F88410BFF34F8FD2F8F1
:1029B000803043F6E074C3F3C900C3F34E335B01C8
:1029C00003EA0406014646EA81750139C2F86052FD
:1029D000F9D2203B13F1200FF2D1BFF34F8F53698F
:1029E00043F480335361BFF34F8FBFF36F8F70BDDC
:1029F00000ED00E0FEE70000214B2248224A70B5BE
:102A0000904237D3214BC11EDA1C121A22F0030266
:102A10008B4238BF00220021FEF76CFA1C4A0023CB
:102A2000C2F88430BFF34F8FD2F8803043F6E074A1
:102A3000C3F3C900C3F34E335B0103EA0406014646
:102A400046EA81750139C2F86C52F9D2203B13F184
:102A5000200FF2D1BFF34F8FBFF36F8FBFF34F8FB4
:102A6000BFF36F8F0023C2F85032BFF34F8FBFF315
:102A70006F8F70BD53F8041B40F8041BC0E700BF04
:102A800064450008C4470020C4470020C447002014
:102A900000ED00E0074BD3F8D81021EA0001C3F89D
:102AA000D810D3F8002122EA0002C3F80021D3F89D
:102AB000003170470044025870B5D0E92443002229
:102AC0004FF0FF359E6804EB42135101D3F8000923
:102AD000002805DAD3F8000940F08040C3F8000967
:102AE000D3F8000B002805DAD3F8000B40F0804043
:102AF000C3F8000B013263189642C3F80859C3F8B3
:102B0000085BE0D24FF00113C4F81C3870BD000020
:102B1000890141F02001016103699B06FCD4122068
:102B2000FFF76EBA10B50A4C2046FEF731FF094B8D
:102B3000C4F89030084BC4F89430084C2046FEF797
:102B400027FF074BC4F89030064BC4F8943010BDF3
:102B5000F445002000000840A843000890460020EB
:102B600000000440B443000870B503780546012B0B
:102B70005CD1434BD0F89040984258D1414B0E2144
:102B80006520D3F8D82042F00062C3F8D820D3F8EB
:102B9000002142F00062C3F80021D3F80021D3F8ED
:102BA000802042F00062C3F88020D3F8802022F019
:102BB0000062C3F88020D3F8803000F0ADFC324BC7
:102BC000E360324BC4F800380023D5F89060C4F8B5
:102BD000003EC02323604FF40413A3633369002B2A
:102BE000FCDA01230C203361FFF70AFA3369DB07B3
:102BF000FCD41220FFF704FA3369002BFCDA00261C
:102C00002846A660FFF758FF6B68C4F81068DB68B9
:102C1000C4F81468C4F81C6883BB1D4BA3614FF053
:102C2000FF336361A36843F00103A36070BD194BD8
:102C30009842C9D1134B4FF08060D3F8D82042F0AE
:102C40000072C3F8D820D3F8002142F00072C3F814
:102C50000021D3F80021D3F8802042F00072C3F89D
:102C60008020D3F8802022F00072C3F88020D3F8AF
:102C70008030FFF70FFF0E214D209EE7064BCDE77A
:102C8000F445002000440258401400400300200294
:102C9000003C30C090460020083C30C0F8B5D0F869
:102CA0009040054600214FF000662046FFF730FFB8
:102CB000D5F8941000234FF001128F684FF0FF30C9
:102CC000C4F83438C4F81C2804EB431201339F4283
:102CD000C2F80069C2F8006BC2F80809C2F8080B14
:102CE000F2D20B68D5F89020C5F8983063621023B3
:102CF0001361166916F01006FBD11220FFF780F958
:102D0000D4F8003823F4FE63C4F80038A36943F410
:102D1000402343F01003A3610923C4F81038C4F81A
:102D200014380B4BEB604FF0C043C4F8103B094B19
:102D3000C4F8003BC4F81069C4F80039D5F89830DD
:102D400003F1100243F48013C5F89820A362F8BD84
:102D50008443000840800010D0F8902090F88A103A
:102D6000D2F8003823F4FE6343EA0113C2F80038B6
:102D7000704700002DE9F84300EB8103D0F8905034
:102D80000C468046DA680FFA81F94801166806F0A9
:102D90000306731E022B05EB41134FF0000194BF95
:102DA000B604384EC3F8101B4FF0010104F11003B4
:102DB00098BF06F1805601FA03F3916998BF06F5B2
:102DC000004600293AD0578A04F158013743490197
:102DD0006F50D5F81C180B430021C5F81C382B1870
:102DE0000127C3F81019A7405369611E9BB3138ACA
:102DF000928B9B08012A88BF5343D8F898209818D3
:102E000042EA034301F140022146C8F898002846EF
:102E100005EB82025360FFF77BFE08EB8900C36875
:102E20001B8A43EA845348341E4364012E51D5F86B
:102E30001C381F43C5F81C78BDE8F88305EB49171B
:102E4000D7F8001B21F40041C7F8001BD5F81C1867
:102E500021EA0303C0E704F13F030B4A2846214659
:102E600005EB83035A60FFF753FE05EB4910D0F8DA
:102E7000003923F40043C0F80039D5F81C3823EAA0
:102E80000707D7E70080001000040002D0F8942064
:102E90001268C0F89820FFF70FBE00005831D0F834
:102EA000903049015B5813F4004004D013F4001F24
:102EB0000CBF0220012070474831D0F89030490102
:102EC0005B5813F4004004D013F4001F0CBF022021
:102ED0000120704700EB8101CB68196A0B68136011
:102EE0004B6853607047000000EB810330B5DD682C
:102EF000AA691368D36019B9402B84BF40231360BB
:102F00006B8A1468D0F890201C4402EB4110013CFD
:102F100009B2B4FBF3F46343033323F0030343EA3E
:102F2000C44343F0C043C0F8103B2B6803F00303D5
:102F3000012B0ED1D2F8083802EB411013F4807F38
:102F4000D0F8003B14BF43F0805343F00053C0F867
:102F5000003B02EB4112D2F8003B43F00443C2F8BD
:102F6000003B30BD2DE9F041D0F8906005460C469D
:102F700006EB4113D3F8087B3A07C3F8087B08D562
:102F8000D6F814381B0704D500EB8103DB685B68B7
:102F90009847FA071FD5D6F81438DB071BD505EB81
:102FA0008403D968CCB98B69488A5A68B2FBF0F6B9
:102FB00000FB16228AB91868DA6890420DD2121AFC
:102FC000C3E90024302383F3118821462846FFF704
:102FD0008BFF84F31188BDE8F081012303FA04F22A
:102FE0006B8923EA02036B81CB68002BF3D0214667
:102FF0002846BDE8F041184700EB81034A0170B54F
:10300000DD68D0F890306C692668E66056BB1A44DB
:103010004FF40020C2F810092A6802F00302012AC6
:103020000AB20ED1D3F8080803EB421410F4807FE3
:10303000D4F8000914BF40F0805040F00050C4F8AC
:10304000000903EB4212D2F8000940F00440C2F834
:1030500000090122D3F8340802FA01F10143C3F850
:10306000341870BD19B9402E84BF402020602068FC
:103070001A442E8A8419013CB4FBF6F440EAC44099
:1030800040F00050C6E700002DE9F843D0F890600A
:1030900005460C464F0106EB4113D3F8088918F09A
:1030A000010FC3F808891CD0D6F81038DB0718D5F3
:1030B00000EB8103D3F80CC0DCF81430D3F800E047
:1030C000DA68964530D2A2EB0E024FF000091A6082
:1030D000C3F80490302383F31188FFF78DFF89F341
:1030E000118818F0800F1DD0D6F834380126A6407C
:1030F000334217D005EB84030134D5F89050D3F850
:103100000CC0E4B22F44DCF8142005EB0434D2F8F0
:1031100000E05168714514D3D5F8343823EA060627
:10312000C5F83468BDE8F883012303FA01F2038986
:1031300023EA02030381DCF80830002BD1D0984742
:10314000CFE7AEEB0103BCF81000834228BF034673
:10315000D7F8180980B2B3EB800FE3D89068A0F1DC
:10316000040959F8048FC4F80080A0EB09089844BA
:10317000B8F1040FF5D818440B4490605360C8E7C9
:103180002DE9F84FD0F8905004466E69AB691E40A7
:1031900016F480586E6103D0BDE8F84FFEF768BCA6
:1031A000002E12DAD5F8003E9B0705D0D5F8003E78
:1031B00023F00303C5F8003ED5F80438204623F079
:1031C0000103C5F80438FEF781FC370505D5204614
:1031D000FFF772FC2046FEF767FCB0040CD5D5F86B
:1031E000083813F0060FEB6823F470530CBF43F458
:1031F000105343F4A053EB6031071BD56368DB68C1
:103200001BB9AB6923F00803AB612378052B0CD104
:10321000D5F8003E9A0705D0D5F8003E23F0030309
:10322000C5F8003E2046FEF751FC6368DB680BB131
:1032300020469847F30200F1BA80B70226D5D4F8A9
:10324000909000274FF0010A09EB4712D2F8003B9B
:1032500003F44023B3F5802F11D1D2F8003B002BAB
:103260000DDA62890AFA07F322EA0303638104EBA9
:103270008703DB68DB6813B139462046984701377E
:10328000D4F89430FFB29B689F42DDD9F00619D57F
:10329000D4F89000026AC2F30A1702F00F0302F496
:1032A000F012B2F5802F00F0CA80B2F5402F09D19C
:1032B00004EB8303002200F58050DB681B6A974211
:1032C00040F0B0803003D5F8185835D5E90303D560
:1032D00000212046FFF746FEAA0303D50121204620
:1032E000FFF740FE6B0303D502212046FFF73AFEAD
:1032F0002F0303D503212046FFF734FEE80203D550
:1033000004212046FFF72EFEA90203D50521204601
:10331000FFF728FE6A0203D506212046FFF722FEAA
:103320002B0203D507212046FFF71CFEEF0103D532
:1033300008212046FFF716FE700340F1A780E90739
:1033400003D500212046FFF79FFEAA0703D50121E0
:103350002046FFF799FE6B0703D502212046FFF7B1
:1033600093FE2F0703D503212046FFF78DFEEE06BF
:1033700003D504212046FFF787FEA80603D50521C3
:103380002046FFF781FE690603D506212046FFF798
:103390007BFE2A0603D507212046FFF775FEEB05C5
:1033A00074D520460821BDE8F84FFFF76DBED4F86C
:1033B00090904FF0000B4FF0010AD4F894305FFA70
:1033C0008BF79B689F423FF638AF09EB4713D3F862
:1033D000002902F44022B2F5802F20D1D3F8002931
:1033E000002A1CDAD3F8002942F09042C3F80029E1
:1033F000D3F80029002AFBDB3946D4F89000FFF708
:1034000087FB22890AFA07F322EA0303238104EBEC
:103410008703DB689B6813B13946204698470BF158
:10342000010BCAE7910701D1D0F80080072A02F109
:1034300001029CBF03F8018B4FEA18283FE704EB19
:10344000830300F58050DA68D2F818C0DCF8082051
:10345000DCE9001CA1EB0C0C00218F4208D1DB68D9
:103460009B699A683A449A605A683A445A6029E7D4
:1034700011F0030F01D1D0F800808C4501F101015A
:1034800084BF02F8018B4FEA1828E6E7BDE8F88F01
:1034900008B50348FFF774FEBDE8084000F07ABBAA
:1034A000F445002008B50348FFF76AFEBDE8084070
:1034B00000F070BB90460020D0F8903003EB411133
:1034C000D1F8003B43F40013C1F8003B7047000003
:1034D000D0F8903003EB4111D1F8003943F40013D8
:1034E000C1F8003970470000D0F8903003EB41116B
:1034F000D1F8003B23F40013C1F8003B70470000F3
:10350000D0F8903003EB4111D1F8003923F40013C7
:10351000C1F8003970470000090100F16043012241
:1035200003F56143C9B283F8001300F01F039A400A
:1035300043099B0003F1604303F56143C3F8802115
:103540001A60704730B50433039C0172002104FBFC
:103550000325C160C0E90653049B0363059BC0E9D2
:103560000000C0E90422C0E90842C0E90A1143632F
:1035700030BD00000022416AC260C0E90411C0E908
:103580000A226FF00101FEF7ABBD0000D0E9043262
:10359000934201D1C2680AB9181D704700207047D4
:1035A000036919600021C2680132C260C269134414
:1035B00082699342036124BF436A0361FEF784BDBD
:1035C00038B504460D46E3683BB162690020131D1F
:1035D0001268A3621344E36207E0237A33B92946F1
:1035E0002046FEF761FD0028EDDA38BD6FF00100DE
:1035F000FBE70000C368C269013BC3604369134431
:1036000082699342436124BF436A4361002383621A
:10361000036B03B11847704770B53023044683F33A
:103620001188866A3EB9FFF7CBFF054618B186F3CD
:103630001188284670BDA36AE26A13F8015B9342C1
:10364000A36202D32046FFF7D5FF002383F311883E
:10365000EFE700002DE9F84F04460E46174698465E
:103660004FF0300989F311880025AA46D4F828B014
:10367000BBF1000F09D141462046FFF7A1FF20B161
:103680008BF311882846BDE8F88FD4E90A12A7EB1E
:10369000050B521A934528BF9346BBF1400F1BD927
:1036A000334601F1400251F8040B914243F8040BF8
:1036B000F9D1A36A403640354033A362D4E90A23E6
:1036C0009A4202D32046FFF795FF8AF31188BD4244
:1036D000D8D289F31188C9E730465A46FDF7E4FB92
:1036E000A36A5E445D445B44A362E7E710B5029CB5
:1036F0000433017203FB0421C460C0E906130023F4
:10370000C0E90A33039B0363049BC0E90000C0E9DE
:103710000422C0E90842436310BD0000026A6FF052
:103720000101C260426AC0E904220022C0E90A2203
:10373000FEF7D6BCD0E904239A4201D1C26822B96F
:10374000184650F8043B0B60704700231846FAE710
:10375000C3680021C2690133C360436913448269AD
:103760009342436124BF436A4361FEF7ADBC00004E
:1037700038B504460D46E3683BB1236900201A1DA5
:10378000A262E2691344E36207E0237A33B929466F
:103790002046FEF789FC0028EDDA38BD6FF0010005
:1037A000FBE7000003691960C268013AC260C269A0
:1037B000134482699342036124BF436A0361002377
:1037C0008362036B03B118477047000070B5302364
:1037D0000D460446114683F31188866A2EB9FFF719
:1037E000C7FF10B186F3118870BDA36A1D70A36A6C
:1037F000E26A01339342A36204D3E16920460439AB
:10380000FFF7D0FF002080F31188EDE72DE9F84F96
:1038100004460D46904699464FF0300A8AF31188C7
:103820000026B346A76A4FB949462046FFF7A0FFD6
:1038300020B187F311883046BDE8F88FD4E90A0734
:103840003A1AA8EB0607974228BF1746402F1BD904
:1038500005F1400355F8042B9D4240F8042BF9D1A3
:10386000A36A40364033A362D4E90A239A4204D3C0
:10387000E16920460439FFF795FF8BF3118846452F
:10388000D9D28AF31188CDE729463A46FDF70CFBD9
:10389000A36A3D443E443B44A362E5E7D0E90423E8
:1038A0009A4217D1C3689BB1836A8BB1043B9B1AC0
:1038B0000ED01360C368013BC360C3691A448369B7
:1038C0009A42026124BF436A036100238362012399
:1038D000184670470023FBE700F086B9014B586A91
:1038E000704700BF000C0040034B002258631A6170
:1038F0000222DA60704700BF000C0040014B00223A
:10390000DA607047000C0040014B5863704700BFFD
:10391000000C0040FEE7000070B51B4B002504467C
:1039200086B058600E468562016300F00BF904F121
:103930001003A560E562C4E904334FF0FF33C4E926
:103940000044C4E90635FFF7C9FF2B46024604F1DF
:1039500034012046C4E9082380230C4A2565FEF77C
:1039600059FB01230A4AE0600092037568467268B9
:103970000192B268CDE90223064BCDE90435FEF78A
:1039800071FB06B070BD00BFB02A0020C043000824
:10399000C543000815390008024AD36A1843D062AB
:1039A000704700BF482800204B6843608B688360E5
:1039B000CB68C3600B6943614B6903628B694362E7
:1039C0000B6803607047000008B53C4B40F2FF7184
:1039D0003B48D3F888200A43C3F88820D3F88820CE
:1039E00022F4FF6222F00702C3F88820D3F888206F
:1039F000D3F8E0200A43C3F8E020D3F808210A43B3
:103A0000C3F808212F4AD3F808311146FFF7CCFF3D
:103A100000F5806002F11C01FFF7C6FF00F5806031
:103A200002F13801FFF7C0FF00F5806002F1540198
:103A3000FFF7BAFF00F5806002F17001FFF7B4FFF5
:103A400000F5806002F18C01FFF7AEFF00F58060A9
:103A500002F1A801FFF7A8FF00F5806002F1C401A0
:103A6000FFF7A2FF00F5806002F1E001FFF79CFF85
:103A700000F5806002F1FC01FFF796FF02F58C7102
:103A800000F58060FFF790FF00F076F90E4BD3F859
:103A9000902242F00102C3F89022D3F8942242F01F
:103AA0000102C3F894220522C3F898204FF0605217
:103AB000C3F89C20054AC3F8A02008BD0044025862
:103AC00000000258CC43000800ED00E01F0008038E
:103AD00008B500F033FBFEF77BFA0F4BD3F8DC2080
:103AE00042F04002C3F8DC20D3F8042122F0400267
:103AF000C3F80421D3F80431084B1A6842F00802D5
:103B00001A601A6842F004021A60FEF721FFBDE84D
:103B10000840FEF7D1BC00BF00440258001802481C
:103B200070470000EFF30983054968334A6B22F0C0
:103B300001024A6383F30988002383F311887047E5
:103B400000EF00E0302080F3118862B60D4B0E4A82
:103B5000D96821F4E0610904090C0A430B49DA60D1
:103B6000D3F8FC2042F08072C3F8FC20084AC2F867
:103B7000B01F116841F0010111602022DA7783F84B
:103B80002200704700ED00E00003FA0555CEACC5F9
:103B9000001000E0302310B583F311880E4B5B68F2
:103BA00013F4006314D0F1EE103AEFF309844FF0F0
:103BB0008073683CE361094BDB6B236684F30988FF
:103BC000FEF7E6F910B1064BA36110BD054BFBE70C
:103BD00083F31188F9E700BF00ED00E000EF00E09B
:103BE0002F04000832040008114BD3F8E82042F0FB
:103BF0000802C3F8E820D3F8102142F00802C3F805
:103C000010210C4AD3F81031D36B43F00803D3636F
:103C1000C722094B9A624FF0FF32DA6200229A61A2
:103C20005A63DA605A6001225A611A60704700BF15
:103C3000004402580010005C000C0040094A08B51E
:103C40001169D3680B40D9B29B076FEA010111617A
:103C500007D5302383F31188FEF7D0F9002383F3CF
:103C6000118808BD000C0040064BD3F8DC2002434D
:103C7000C3F8DC20D3F804211043C3F80401D3F8BF
:103C800004317047004402583A4B4FF0FF31D3F8EB
:103C9000802062F00042C3F88020D3F8802002F038
:103CA0000042C3F88020D3F88020D3F88420C3F8E2
:103CB0008410D3F884200022C3F88420D3F8840031
:103CC000D86F40F0FF4040F4FF0040F4DF4040F088
:103CD0007F00D867D86F20F0FF4020F4FF0020F469
:103CE000DF4020F07F00D867D86FD3F888006FEAF4
:103CF00040506FEA5050C3F88800D3F88800C0F3F2
:103D00000A00C3F88800D3F88800D3F89000C3F8FD
:103D10009010D3F89000C3F89020D3F89000D3F817
:103D20009400C3F89410D3F89400C3F89420D3F807
:103D30009400D3F89800C3F89810D3F89800C3F80B
:103D40009820D3F89800D3F88C00C3F88C10D3F8DF
:103D50008C00C3F88C20D3F88C00D3F89C00C3F8F7
:103D60009C10D3F89C10C3F89C20D3F89C3000F032
:103D7000B9B900BF0044025808B50122534BC3F83B
:103D80000821534BD3F8F42042F00202C3F8F42088
:103D9000D3F81C2142F00202C3F81C210222D3F8FE
:103DA0001C314C4BDA605A689104FCD54A4A1A60BF
:103DB00001229A60494ADA6000221A614FF44042B7
:103DC0009A61444B9A699204FCD51A6842F4807255
:103DD0001A603F4B1A6F12F4407F04D04FF48032C8
:103DE0001A6700221A671A6842F001021A60384BFB
:103DF0001A685007FCD500221A611A6912F03802BD
:103E0000FBD1012119604FF0804159605A67344A53
:103E1000DA62344A1A611A6842F480321A602C4B12
:103E20001A689103FCD51A6842F480521A601A6825
:103E30009204FCD52C4A2D499A6200225A631963D8
:103E400001F57C01DA6301F2E71199635A64284AAB
:103E50001A64284ADA621A6842F0A8521A601C4BA7
:103E60001A6802F02852B2F1285FF9D148229A610B
:103E70004FF48862DA6140221A621F4ADA641F4AEC
:103E80001A651F4A5A651F4A9A6532231E4A1360F3
:103E9000136803F00F03022BFAD10D4A136943F0A4
:103EA00003031361136903F03803182BFAD14FF0A1
:103EB0000050FFF7D9FE4FF08040FFF7D5FE4FF0DE
:103EC0000040BDE80840FFF7CFBE00BF00800051B2
:103ED000004402580048025800C000F002000001EF
:103EE0000000FF01008890082220400063020901C1
:103EF000470E0508DD0BBF01200000200000011067
:103F00000910E00000010110002000524FF0B04203
:103F100008B5D2F8883003F00103C2F8883023B125
:103F2000044A13680BB150689847BDE80840FFF792
:103F300031BE00BF444700204FF0B04208B5D2F870
:103F4000883003F00203C2F8883023B1044A936832
:103F50000BB1D0689847BDE80840FFF71BBE00BF13
:103F6000444700204FF0B04208B5D2F8883003F043
:103F70000403C2F8883023B1044A13690BB15069B5
:103F80009847BDE80840FFF705BE00BF4447002042
:103F90004FF0B04208B5D2F8883003F00803C2F8F9
:103FA000883023B1044A93690BB1D0699847BDE8C2
:103FB0000840FFF7EFBD00BF444700204FF0B0427C
:103FC00008B5D2F8883003F01003C2F8883023B166
:103FD000044A136A0BB1506A9847BDE80840FFF7DE
:103FE000D9BD00BF444700204FF0B04310B5D3F80F
:103FF000884004F47872C3F88820A30604D5124AD6
:10400000936A0BB1D06A9847600604D50E4A136BC9
:104010000BB1506B9847210604D50B4A936B0BB13B
:10402000D06B9847E20504D5074A136C0BB1506C6E
:104030009847A30504D5044A936C0BB1D06C9847FC
:10404000BDE81040FFF7A6BD444700204FF0B04345
:1040500010B5D3F8884004F47C42C3F88820620588
:1040600004D5164A136D0BB1506D9847230504D53E
:10407000124A936D0BB1D06D9847E00404D50F4AF6
:10408000136E0BB1506E9847A10404D50B4A936E82
:104090000BB1D06E9847620404D5084A136F0BB178
:1040A000506F9847230404D5044A936F0BB1D06F27
:1040B0009847BDE81040FFF76DBD00BF44470020A2
:1040C00008B50348FDF770F8BDE80840FFF762BD8A
:1040D000D823002008B5FFF7B1FDBDE80840FFF781
:1040E00059BD0000062108B50846FFF715FA06215C
:1040F0000720FFF711FA06210820FFF70DFA062125
:104100000920FFF709FA06210A20FFF705FA062120
:104110001720FFF701FA06212820FFF7FDF90921F2
:104120007A20FFF7F9F907213220FFF7F5F90C2182
:104130005220BDE80840FFF7EFB9000008B5FFF7CF
:10414000A3FD00F00DF8FDF747FAFDF71FFCFDF7A2
:10415000F1FAFFF7E5FCBDE80840FFF7BDBB000042
:104160000023054A19460133102BC2E9001102F160
:104170000802F8D1704700BF4447002010B501394C
:104180000244904201D1002005E0037811F8014F6C
:10419000A34201D0181B10BD0130F2E7034611F80D
:1041A000012B03F8012B002AF9D1704753544D33EA
:1041B0003248373F3F3F0053544D3332483733780E
:1041C0002F3732780053544D3332483734332F373A
:1041D00035332F373530000001105A0003105900D5
:1041E0000120580003205600009600000000000047
:1041F00000000000000000000000000000000000BF
:10420000000000009915000885150008C115000878
:10421000AD150008B9150008A5150008911500088E
:104220007D150008CD15000800000000B11600083B
:104230009D160008D9160008C5160008D1160008FA
:10424000BD160008A916000895160008E516000816
:1042500000000000010000000000000063300000CA
:104260005C420008A0280020B02A0020417264753A
:1042700050696C6F740025424F415244252D424CC9
:10428000002553455249414C250000000200000022
:1042900000000000D118000841190008400040004B
:1042A0006043002070430020020000000000000076
:1042B0000300000000000000891900080000000051
:1042C00010000000804300200000000001000000FA
:1042D00000000000F4450020010102005524000800
:1042E0006523000801240008E523000843000000BE
:1042F000F442000809024300020100C03209040030
:104300000001020201000524001001052401000142
:10431000042402020524060001070582030800FFA9
:1043200009040100020A0000000705010240000024
:104330000705810240000000120000004043000811
:10434000120110010200004009124157000201024F
:10435000030100000403090425424F415244250093
:10436000594A5541565F413653455F48373433000B
:10437000303132333435363738394142434445469B
:104380000000000000000000E51A00089D1D000864
:10439000491E0008400040002C4700202C47002008
:1043A000010000003C4700208000000040010000A8
:1043B00008000000000100000010000008000000DC
:1043C0006D61696E0069646C650000000100802AFF
:1043D00000000000AAAAAAAA01000024FFFF000012
:1043E0000000000000A00A00000000000000000023
:1043F000AAAAAAAA00000000FFFF00000000000017
:10440000000000000000004000000000AAAAAAAAC4
:1044100000000040FFFF000000000000000000005E
:104420000000100000040000AAAAAAAA00000000D0
:10443000FFFF000000000000000000004085164063
:1044400000800000AAAAAAAA40451500FFFF0000AC
:1044500000000070070000000000000000000000E5
:10446000AAAAAAAA00000000FFFF000000000000A6
:10447000000000000100000001000000AAAAAAAA92
:1044800000000000FFFF000000000000000000002E
:104490000000000000000000AAAAAAAA0000000074
:1044A000FFFF00000000000000000000000000000E
:1044B00000000000AAAAAAAA00000000FFFF000056
:1044C00000000000000000000000000000000000EC
:1044D000AAAAAAAA00000000FFFF00000000000036
:1044E000000000000000000000000000AAAAAAAA24
:1044F00000000000FFFF00000000000000000000BE
:10450000750400000000000000001E000000000014
:10451000FF000000B82A0020D8230020000000007F
:10452000AC41000883040000B741000850040000BB
:10453000C541000800960000000008009600000039
:1045400000080000040000005443000800000000C0
:10455000000000000000000000000000000000005B
:044560000000000057
:00000001FF
